:1000000000308A00D128000016308400000803194F
:10001000182801308D008C018C0B0C288D0B0B28BF
:100020004A308C008C0B122800000000800B09283D
:10003000DB28970183160614861083128610213060
:100040008C008C0B212883160610831206100630B4
:100050008C008C0B29280000831686148312861CC2
:100060002C2896011608073C031C52288316861478
:1000700083128618362815080139003A031D4228D4
:10008000061043280614831606108312150801393A
:1000900097070310950C831686148312861C4B2831
:1000A000960A322883168614831286185228170857
:1000B000FF3A0139003A031D5F2806106028061434
:1000C0008316061086148312861868288316622801
:1000D00069288316861483128618692806148316E5
:1000E00006108614831286187728831671287828BC
:1000F000831606148312E0289601160203188D2831
:10010000831686148312861C8A288316061483128B
:1001100006188B289601960A7D288316861483126A
:1001200086188D2883160614831206188D288316C8
:1001300086148312861C9728950196011608073CA1
:10014000031CBD288316861483128618A228031068
:10015000950C8316061400308312061801308C00AB
:100160000C0C8C0103188C170C089504831686144C
:100170008312861CB628960A9E2815088D00003426
:1001800083160510831205148316051083120510BB
:1001900021308C008C0BCA2883160510831205149D
:1001A000FC2884011F3083059101940102309500E1
:1001B000FA3096000428950BD828F43095001928B9
:1001C000E83083160317FF00831203137C200D0809
:1001D0009100023083160317FF00831203137C2063
:1001E0000D088F00023083160317FF0083120313DC
:1001F0007C200D089000C028111E072983160511C8
:100200008312051583168511831285110F29831614
:100210008511831285158316051183120511E028B7
:02022000630079
:02400E00F93F78
:00000001FF
